:20000000A2C0CAC2F8C2B8C025C3B6C0B5C0B4C0B3C0B2C0B1C0B0C0AFC0AEC0ADC0ACC0FD
:20002000ABC0AAC0A9C073C178C174C172C184C173C175C176C177C178C179C17AC17BC1A5
:200040007DC17EC17FC180C181C182C183C184C185C186C187C199C19EC19AC198C1A8C1E9
:2000600099C19BC19CC1BBC19CC19DC19EC19FC1A1C1A2C1A3C1E4C1A3C1A4C1A5C1A6C113
:20008000A7C1A8C1A9C1AAC1ACC1ADC1AEC1AFC1B0C1B1C1B2C1B3C1B4C1B5C1B6C1B7C15C
:2000A000B8C1B9C1BAC1BBC1BCC1BDC1BEC1BFC1C0C1C1C1C2C1C3C1C5C1C6C1C7C1C8C134
:2000C000C9C1CAC1CBC1CCC1CDC1CEC1CFC1E6C1EBC1E7C1E5C1F5C1E6C1E8C1E9C108C22A
:2000E000E9C1EAC1EBC1ECC1EEC1EFC1F0C131C2F0C1F1C1F2C1F3C1F4C1F5C1F6C1F7C1AB
:20010000F9C1FAC1FBC1FCC1FDC1FEC1FFC100C201C202C203C204C205C206C207C208C2BE
:2001200009C20AC20BC20CC20DC20EC20FC210C212C213C214C215C216C217C218C219C28F
:200140001AC21BC21CC211241FBECFEDCDBF10E0A0E6B0E0E4ECF7E002C005900D92A23633
:20016000B107D9F710E0A2E6B0E001C01D92A736B107E1F7B4D224C343CFC09AC19AC29A82
:20018000C39AC49AC59AC69AC79A0895C298C198C0980895C398C198C0980895C398C298E1
:2001A000C0980895C398C298C1980895C398C298C198C0980895C498C198C0980895C49896
:2001C000C298C0980895C498C298C1980895C498C298C198C0980895C498C398C098089574
:2001E000C498C398C1980895C498C398C198C0980895C498C398C2980895C498C398C2988E
:20020000C0980895C498C398C298C1980895C498C398C298C198C0980895C598C198C09875
:200220000895C598C298C0980895C598C298C1980895C598C298C198C0980895C598C3980B
:20024000C0980895C598C398C1980895C598C398C198C0980895C598C398C2980895C598E9
:20026000C398C298C0980895C598C398C298C1980895C598C398C298C198C0980895C5980F
:20028000C498C0980895C598C498C1980895C598C498C198C0980895C598C498C2980895A7
:2002A000C598C498C298C0980895C598C498C298C1980895C598C498C298C198C0980895CC
:2002C000C598C498C3980895C598C498C398C0980895C598C498C398C1980895C598C498A1
:2002E000C398C198C0980895C098C198C298C398C498C598C698C798089580916200E82F52
:20030000F0E0E831F10578F5ED5EFF4F099435DF2AC0C098C19827C0C298C09824C0C298D5
:20032000F9CF34DF20C0C3981EC0C398F6CFC398F1CF30DF18C0C398C29815C02FDF13C03C
:2003400031DF11C033DF0FC0C4980DC0C498E5CFC498E0CF30DF07C0C498EECF30DF03C0D6
:2003600032DF01C034DF80916200883110F010926200089580916300E82FF0E0EC33F1055B
:2003800008F075C0E55DFF4F0994F7DE70C0C098C1986DC0C298C0986AC0C298F9CFF6DE4E
:2003A00066C0C398F8CFC398F3CFF4DE60C0C398C2985DC0F3DE5BC0F5DE59C0F7DE57C050
:2003C000C498E9CFC498E4CFF6DE51C0C498F0CFF6DE4DC0F8DE4BC0FADE49C0C498C398A0
:2003E00046C0FADE44C0FCDE42C0FEDE40C001DF3EC003DF3CC006DF3AC009DF38C0C5988B
:2004000036C0C598C8CFC598C3CF07DF30C0C598CFCF07DF2CC009DF2AC00BDF28C0C5985F
:20042000DECF0CDF24C00EDF22C010DF20C013DF1EC015DF1CC018DF1AC01BDF18C0C59802
:20044000C49815C01CDF13C01EDF11C020DF0FC023DF0DC025DF0BC028DF09C02BDF07C0C2
:200460002FDF05C031DF03C034DF01C037DF809163008C3338F0809162008F5F80936200BB
:2004800010926300089580916400E82FF0E0EC33F10508F075C0E959FF4F09946EDE70C073
:2004A000C098C1986DC0C298C0986AC0C298F9CF6DDE66C0C398F8CFC398F3CF6BDE60C047
:2004C000C398C2985DC06ADE5BC06CDE59C06EDE57C0C498E9CFC498E4CF6DDE51C0C49846
:2004E000F0CF6DDE4DC06FDE4BC071DE49C0C498C39846C071DE44C073DE42C075DE40C07F
:2005000078DE3EC07ADE3CC07DDE3AC080DE38C0C59836C0C598C8CFC598C3CF7EDE30C006
:20052000C598CFCF7EDE2CC080DE2AC082DE28C0C598DECF83DE24C085DE22C087DE20C00F
:200540008ADE1EC08CDE1CC08FDE1AC092DE18C0C598C49815C093DE13C095DE11C097DEF5
:200560000FC09ADE0DC09CDE0BC09FDE09C0A2DE07C0A6DE05C0A8DE03C0ABDE01C0AEDE2D
:20058000809164008C3338F0809163008F5F809363001092640008951F920F920FB60F92CC
:2005A00011242F933F938F939F93EF93FF93809160008230A8F081E0809360008091620008
:2005C0008F5F80936200109266001092650080ED97E022E330E0F9013197F1F70197D9F79E
:2005E000FF91EF919F918F913F912F910F900FBE0F901F9018951F920F920FB60F921124B7
:200600002F933F938F939F93EF93FF93809160008230A8F081E080936000809163008F5FED
:2006200080936300109266001092650080ED97E022E330E0F9013197F1F70197D9F7FF919A
:20064000EF919F918F913F912F910F900FBE0F901F9018951F920F920FB60F9211248F93C4
:20066000809164008F5F809364008F910F900FBE0F901F90189580E090E094980196883CC2
:200680009105D9F7949A089580E090E095980196883C9105D9F7959A089580E090E09698A1
:2006A0000196883C9105D9F7969A0895E4DFECDFF4CF80E090E0949A0196883C9105D9F79C
:2006C00080E090E0959A0196883C9105D9F780E090E0969A0196883C9105D9F70895CF929B
:2006E000DF92EF92FF920F931F93CF93DF9387B38FEF87BB81B3806781BB81B38C7F81BB83
:2007000082B38C6082BB8BB7806C8BBF85B78C6085BF789488B3806788BB88B38FEF88BB2A
:2007200032E0C32E2BE0D22E90E4E92E02E11AE783E0F82E80916000843079F4D5DDC0E0CF
:20074000D0E0B4DF2196C83CD105D9F7C0E0D0E0B0DF2196C83CD105D9F780916000882399
:20076000A1F080916000833080F480916500909166000196909366008093650010926400B5
:2007800089B78F7B89BFC09260008091650090916600805A9F4051F4DEBCE9BE1BBD0ABD3A
:2007A0001092660010926500F0926000E6DC6BDE74DFE3DCDFDD68DFE0DC9FDD5CDFBACF2C
:0607C000F894FFCF0400D5
:00000001FF
